:020000040800F2
:101000000080002079400008C14D0008C54D00084F
:10101000C94D0008CD4D0008D14D0008000000006A
:10102000000000000000000000000000D54D000896
:10103000D94D000800000000DD4D0008E14D00081A
:10104000C1400008C1400008C1400008C14000087C
:10105000C1400008C1400008C1400008C14000086C
:10106000C1400008C1400008C1400008E54D00082B
:10107000C1400008C14000080D4E0008C1400008F2
:101080004D4E0008C1400008C1400008C1400008A2
:10109000C1400008C1400008C1400008C14000082C
:1010A000054F0008394F0008214F0008C1400008D3
:1010B000C1400008514F0008C1400008C14000086D
:1010C000C1400008C1400008C1400008C1400008FC
:1010D000C14000084D4F0008C1400008C140000851
:1010E000754F0008C1400008C14000080000000022
:1010F00000000000000000000000000000000000F0
:1011000000000000C1400008C140000800000000CD
:10111000C1400008C14000080000000000000000BD
:10112000C1400008C1400008C1400008C14000089B
:1011300000000000000000000000000000000000AF
:10114000000000000000000000000000C140000896
:101150000000000000000000ED4E0008C140000843
:10116000000000000000000000000000C140000876
:101170004FF0FF0C1CEAD0521EBF1CEAD15392EA7A
:101180000C0F93EA0C0F6FD01A4480EA010C400256
:1011900018BF5FEA41211ED04FF0006343EA5010B0
:1011A00043EA5111A0FB01310CF00040B1F5000FF2
:1011B0003EBF490041EAD3715B0040EA010062F1A1
:1011C0007F02FD2A1DD8B3F1004F40EBC25008BF8B
:1011D00020F00100704790F0000F0CF0004C08BFA9
:1011E00049024CEA502040EA51207F3AC2BFD2F176
:1011F000FF0340EAC250704740F400004FF0000384
:10120000013A5DDC12F1190FDCBF00F000407047BD
:10121000C2F10002410021FA02F1C2F1200200FAFB
:1012200002FC5FEA310040F1000053EA4C0308BFC2
:1012300020EADC70704792F0000F00F0004C02BF13
:10124000400010F4000F013AF9D040EA0C0093F08E
:10125000000F01F0004C02BF490011F4000F013BE8
:10126000F9D041EA0C018FE70CEAD15392EA0C0F56
:1012700018BF93EA0C0F0AD030F0004C18BF31F0C1
:10128000004CD8D180EA010000F00040704790F097
:10129000000F17BF90F0004F084691F0000F91F03B
:1012A000004F14D092EA0C0F01D142020FD193EA01
:1012B0000C0F03D14B0218BF084608D180EA010089
:1012C00000F0004040F0FE4040F40000704740F065
:1012D000FE4040F44000704780F0004002E000BF54
:1012E00081F0004142001FBF5FEA410392EA030F11
:1012F0007FEA226C7FEA236C6AD04FEA1262D2EB5B
:101300001363C1BFD218414048404140B8BF5B425F
:10131000192B88BF704710F0004F40F4000020F0F8
:101320007F4018BF404211F0004F41F4000121F00E
:101330007F4118BF494292EA030F3FD0A2F1010258
:1013400041FA03FC10EB0C00C3F1200301FA03F196
:1013500000F0004302D5494260EB4000B0F5000FB9
:1013600013D3B0F1807F06D340084FEA310102F178
:101370000102FE2A51D2B1F1004F40EBC25008BF2A
:1013800020F0010040EA03007047490040EB0000F4
:10139000013A28BFB0F5000FEDD2B0FA80FCACF1F5
:1013A000080CB2EB0C0200FA0CF0AABF00EBC25022
:1013B00052421843BCBFD0401843704792F0000F10
:1013C00081F4000106BF80F400000132013BB5E763
:1013D0004FEA41037FEA226C18BF7FEA236C21D0D9
:1013E00092EA030F04D092F0000F08BF084670473E
:1013F00090EA010F1CBF0020704712F07F4F04D10C
:10140000400028BF40F00040704712F100723CBF1E
:1014100000F50000704700F0004343F0FE4040F448
:10142000000070477FEA226216BF08467FEA236306
:101430000146420206BF5FEA412390EA010F40F4F1
:10144000800070474FF0000304E000BF10F000433D
:1014500048BF40425FEA000C08BF704743F0964324
:1014600001464FF000001CE050EA010208BF70473F
:101470004FF000030AE000BF50EA010208BF7047C6
:1014800011F0004302D5404261EB41015FEA010CDB
:1014900002BF84460146002043F0B64308BFA3F1D3
:1014A0008053A3F50003BCFA8CF2083AA3EBC253B5
:1014B00010DB01FA02FC634400FA02FCC2F12002D4
:1014C000BCF1004F20FA02F243EB020008BF20F00B
:1014D0000100704702F1200201FA02FCC2F1200271
:1014E00050EA4C0021FA02F243EB020008BF20EA66
:1014F000DC7070474FF0FF3C06E000BF4FF0010C7E
:1015000002E000BF4FF0010C4DF804CD4FEA40025D
:101510004FEA41037FEA226C18BF7FEA236C11D0A7
:1015200001B052EA530C18BF90EA010F58BFB2EB5A
:10153000030088BFC81738BF6FEAE17018BF40F0DA
:10154000010070477FEA226C02D15FEA402C05D18E
:101550007FEA236CE4D15FEA412CE1D05DF8040B13
:10156000704700BF844608466146FFE70FB5FFF7A6
:10157000C9FF002848BF10F1000F0FBD4DF808ED5E
:10158000FFF7F4FF0CBF012000205DF808FB00BF4F
:101590004DF808EDFFF7EAFF34BF012000205DF8A9
:1015A00008FB00BF4DF808EDFFF7E0FF94BF0120F6
:1015B00000205DF808FB00BF4DF808EDFFF7D2FFF3
:1015C00094BF012000205DF808FB00BF4DF808ED36
:1015D000FFF7C8FF34BF012000205DF808FB00BF03
:1015E0004FEA4002B2F1FE4F0FD34FF09E03B3EB30
:1015F00012620DD94FEA002343F0004310F0004F70
:1016000023FA02F018BF404270474FF000007047C5
:1016100012F1610F01D1420205D110F0004008BF64
:101620006FF0004070474FF00000704742000ED24C
:10163000B2F1FE4F0BD34FF09E03B3EB126209D40D
:101640004FEA002343F0004323FA02F070474FF0C3
:101650000000704712F1610F01D1420202D14FF038
:10166000FF3070474FF00000704700BF53B94AB9D0
:10167000002908BF00281CBF4FF0FF314FF0FF309A
:1016800000F00CB8ADF1080C6DE904CE04F0D4FB09
:10169000DDF804E0DDE9022304B07047704700BFC5
:1016A00010B5054C237833B9044B13B10448AFF39C
:1016B00000800123237010BD6A0800200000000094
:1016C0006061000808B5034B1BB103490348AFF341
:1016D000008008BD000000006C0800206061000868
:1016E000A449A5480B68CA6F00882DE9F04FD21AAB
:1016F00092B2A24C5509904283B02280658062D29A
:101700009F48008890425ED99E480022028004F1E2
:101710004006204601E051F8083F4A68D21A92B2CA
:1017200095422CBF0022012240F8042F8642F2D1BC
:10173000A56BA368D4F818A0D4F804E06169A26A84
:10174000D4F824B02069D4F820800193AE00656BF2
:10175000E768D4F82CC083EA0A0946EAC50689EA94
:1017600002098EEA010585EA0B054FEA8909E3695A
:10177000009349EAC509256C236B354380EA0806C6
:101780005E4049EA0609E66B009B45EA4605EEB273
:1017900087EA03057C4B85EA0C0549EA450593F881
:1017A0000090EDB2B9F1000F10D0DFF8E09199F898
:1017B0000090B9F1000F0FD1AE4211D0B4F8503003
:1017C0000133A4F8503003B0BDE8F08FDFF8BC91CE
:1017D00099F80030002B60D0C6F10F06F6B2EBE7A7
:1017E000684BB4F8465000261E80019B5B0243EA1A
:1017F0008E2343EA0C0343EA072343EAC01301356F
:1018000043EA81130099A4F8465043EA4A13256B32
:1018100043EA0113012D43EAC80308BF5C4E43EAC3
:101820008B0343EA420208BF35702F2A1BDD94F870
:101830004830002B5BD1574D2A78002AC3D0564B35
:101840001B78002BBFD1504B1B78002BBBD094F8DA
:101850004B30934253D0042A84F84B205AD90123A9
:1018600084F84930AFE7531E2E2B0FD9002AE2D15E
:1018700094F84A304949012B08BF84F84820454A6A
:1018800000230B80137084F849309CE7434B414D93
:101890000021D2B219802A70D1E703F0E3FCC0B175
:1018A00094F844300133DBB2642B84F8443010D90F
:1018B000012389F80030D4E901E30193E36900933F
:1018C000D4E90370D4E9051AD4E9088BD4E90A2CC9
:1018D00082E7D4E901E30193E3690093D4E903705B
:1018E000D4E9051AD4E9088BD4E90A2C5FE72B4820
:1018F0002849028000230B7084F8493063E7042AEA
:1019000008D994F849300133DBB2052B84F849300B
:101910007FF659AF0023013A84F84930142A0FD8D2
:10192000DFE802F00B7E7A76720E6B64605C0E5418
:1019300046200E0E0E0E0E191400194B01221A70BD
:10194000184A2978117000232B703CE7164A174B70
:1019500012781A70F4E7144B144A1B78C3F1010390
:101960001370EDE7002240F6FF6384F84C20A4F8E2
:101970004E30E5E7600700204C070020DC03002024
:10198000D0030020DE060020AC060020ED0600207B
:10199000D8060020040700209706002098060020A3
:1019A000B2060020050700208C05002067000020FB
:1019B00094F84A3001214FF460628B4284F84C1055
:1019C000A4F84E20BCD184F84830B9E700F052FBAF
:1019D000154B164A1B7801331370B1E7144B0122E3
:1019E0001A70ADE7124B00221A70A9E70E49114B8D
:1019F0000120002208701A70A2E70B490D4B00204D
:101A0000012208701A709BE7084B05221A7097E7AD
:101A1000064B04221A7093E7044B03221A708FE7D7
:101A2000024B02221A708BE78C050020B2060020C0
:101A30008D0500206700002030B52F4DB5F84E30E1
:101A4000002B3FD000221846A5F84E201A0A82EA41
:101A500013125340DB4303F00F0343EA0013274AFA
:101A6000AB6503F00F001913145C515C244844EA81
:101A7000C134C3F30321C3F30313515CD35C214A84
:101A800092F800E044EA812444EA431405EB8E0313
:101A9000802200EB8E00EC655A66043013214FF073
:101AA000010C0CFA01F32340CB4083EAD212013936
:101AB000D2014B1C40F8042FF3D105EB8E05002317
:101AC0002B6630BD104B1B785BB103460F2240FAEA
:101AD00002F1012908D0013A082AF8D100226A65EA
:101AE000B4E74FF6FF70F0E7083A40FA02F343EA32
:101AF00042206A6583B2A9E7DC0300207861000810
:101B00003C040020D30300209706002030B5039C3E
:101B100084460AE08C4513DD9C420FD0B1EB6E0F7A
:101B20000DD0AC450EDC04462A4602EB010EE0184F
:101B300094454FEA6E054FEA6000EBDB204630BD6E
:101B4000184630BD691C0346EFE700BF0346401A44
:101B500048BFC81A704700BF034A00235362536A44
:101B60008342FCD3704700BF005001400B4A4FF442
:101B70006153002151629362536900EB800043F08E
:101B8000010353614000536A8342FCD39023936264
:101B9000536943F001035361704700BF0050014097
:101BA000F0B5074683B00E4614461D4672B6684629
:101BB00002F0B8FE694638468DF8066000958DF84B
:101BC000054002F051FE62B603B0F0BDBFF34F8F87
:101BD0000549064BCA6802F4E0621343CB60BFF3C9
:101BE0004F8F00BFFDE700BF00ED00E00400FA05E5
:101BF00003468A1A0069996810B51C6A1A6001FBCD
:101C00000201A1421961C4BF21461C6164428C4299
:101C10009869C4BF1C612146DC68101A04FB00F0FF
:101C20005C68586104FB02005C6A0844A042C3E996
:101C30000620C4BFDC61204664428442C4BFDC612C
:101C40002046FFF703FC10BD03460069511A1A6ACB
:101C50000844904210B51861C4BF10461A61524240
:101C60008242C4BF10461A615A68196002FB01FC27
:101C70009A69114C8A1AC3E90521996801FB00F0A1
:101C80000E4984FB0C4E81FB00414FEAEC7CC017EF
:101C9000C0EB2130CCEB6E1CD968604401FB020222
:101CA000586ADA61824202DC4042824201DAD8613B
:101CB00010BD104610BD00BF1F85EB51AD8BDB681A
:101CC00070B5C04CC04DB8222968204682B003F0E0
:101CD00019FA627CA37CE17C207EA2F10102B2FAB7
:101CE00082F2520984F8B820627DA3F10103B3FAAD
:101CF00083F3A2F101025B09B2FA82F201294FEAF1
:101D0000521284F8B930E37D08BF84F8BA106A71C2
:101D1000217DA27D042B28BF0223A1F10101A2F1A4
:101D20000102B1FA81F1B2FA82F2EB71A0F108037B
:101D300049095209282B2971AA7151D8A0F1180319
:101D4000182B40F24D81A0F10C030B2B40F259816E
:101D5000A0F10803032B40F2658128899B4BD862D0
:101D6000637EA3F13202642A44D8994AAB81A2FB74
:101D700003235B0803F10A02EB812A82A37E217F01
:101D8000627FE07E287503EB8303A1F10101A2F1DC
:101D90000102DB00B1FA81F1B2FA82F2143349098F
:101DA000520902206B8284F8BB1084F8BC2002F038
:101DB00051F86378002B46D1688A4FF4FA73009388
:101DC00040F6B8324FF47A734FF49671FFF79EFEE7
:101DD00094F8B130688693B984F8C53002B070BD0C
:101DE0007A4A41F270736B81D362637EA3F132024F
:101DF000642ABAD996225523AA81EB81BEE794F8CA
:101E0000B33094F8B22094F8B40094F8B710286472
:101E100003EB830302EB820203EB8303DB0002EBA1
:101E200082020120D200AB636A4B84F8C5006A636A
:101E300094F8B50094F8B62001FB03F3C5E911024C
:101E4000EB6502B070BDA07F0B2888BF052002F0B3
:101E500001F894F8202094F82130E17F94F82300D1
:101E6000287702F277125200EA8294F8222003F2D5
:101E70006B335B0002F25E522B836A8394F8263048
:101E800094F82520A3F10103FA32B3FA83F3EA832D
:101E900094F828205B09A1F10101B1FA81F184F8DD
:101EA000BF30531F142B4FEA511194F8293084F896
:101EB000BD1094F8241098BF85F820205A1E092AD6
:101EC000A1F1010194F82A2098BF85F82130B1FAD8
:101ED00081F14909531E84F8BE10082B4FF0000110
:101EE00084F8C0101ED8C2EB4213C2EB83035B0020
:101EF000063BDBB2C82B85F8222000F29F8085F8D4
:101F000023309AB2A98C314E607E1144A984E98CA9
:101F10001144E984716C0B437364131802EB500293
:101F2000AB81EA8194F82B30A3F14602462A98BF90
:101F300085F8283094F82C305A1E622A04D85B00A9
:101F400001226B8584F8C12094F82D305A1E092A8D
:101F500098BF85F82C3094F82E30092B06D8042B26
:101F60000CD8DFE803F0037D790B70001A4A0023D8
:101F7000012184F8C23084F8C330117094F82F30F6
:101F8000688A164A297DA3F10103B3FA83F35B093A
:101F9000B0F5967F84F8C4303CBF002385F82D301F
:101FA0002023B3FBF1F1A2FB0032094B5209B2FB33
:101FB000F1F2EA85A3FB0023DB08B3FBF1F32B86E8
:101FC000FBE600BFD404002000000020002C0140EC
:101FD000ABAAAAAAA0860100240400201F85EB5109
:101FE00040F6B8330093302241F270731821FFF7A6
:101FF0008DFD0346207E2B81A0F10C030B2B3FF6B9
:10200000A7AE41F270730093182242F6E0630C21F0
:10201000FFF77CFD0346207E2B81A0F10803032BF4
:102020003FF69BAE42F228330093102244F25063F5
:102030000721FFF76BFD80B228818FE6C822134687
:1020400085F823205EE70949094A01230B70002126
:10205000117084F8C23091E7012384F8C3308DE712
:10206000034A012384F8C230137087E72604002056
:102070002404002000B52148214B90F8B8C090F806
:10208000B92090F8BA1093F864E080F801E0ACF160
:10209000010CA2F10102A1F10101BCFA8CFCB2FA1F
:1020A00082F2B1FA81F14FEA5C1C5209490980F8C9
:1020B00011C08274C1741A7993F805C0997993F8A4
:1020C00007E080F817E0A2F10102ACF1010CA1F1E8
:1020D0000101B2FA82F2BCFA8CFCB1FA81F1520928
:1020E00049094FEA5C1C0275817580F815C01A68B1
:1020F0005DF804EBB82102F0A9BF00BFD4040020B2
:102100000000002000B5124A92F8CC10B2F89831C5
:10211000D2F8C80002EB410C0131C9B26329BCF806
:10212000D0E0ACF8D030184484BF002382F8CC3023
:10213000084B98BF82F8CC10A0EB0E00C2F8C80084
:10214000A3FB0030C0F34F10A2F89A015DF804FB26
:10215000D40400201F85EB5108B502F017FF0E4B89
:1021600093F865203AB140B90C4A92F89C3101339A
:1021700082F89C3108BD0028F6D1084A93F8661011
:1021800092F89D310133DBB2994282F89D31F1D250
:10219000002382F89C3108BD00000020D4040020F8
:1021A00038B5284C94F86730012B3BD094F8683050
:1021B000254D5A1E12F0FF0222D084F8682003F049
:1021C000010384F8653072B695F89F312BB362B67F
:1021D00002F0F8FED5F8A021E16E40F2A4639A4225
:1021E00084BF012384F8693094F8683005EB430319
:1021F000002285F89C2185F8A421A3F8A61138BDFA
:102200000123062284F8682085F89E3184F8653021
:1022100072B695F89F31002BD9D194F8680003F07D
:1022200051FBD4E794F86820074D0132D2B2062A58
:1022300099BF84F8682002F0010384F8683085F8BB
:102240009E31BEE700000020D40400201B4AD36862
:1022500023F0010310B5D360FFF7A2FF1849194C12
:10226000CB6EB4F8B40194F8C42003EB43030344E9
:102270009808C866C2B991F87020580912FB00F29C
:1022800092B291F86910A4F8B821C2EBD303A4F874
:10229000BA3181B1D4F8BC3142F20F7293429CBF83
:1022A0000133C4F8BC3110BD94F8B62100FB02F232
:1022B000C2F38F12E5E702F07DFEEBE70054014028
:1022C00000000020D404002070B5254ED6F8A031BF
:1022D0007D2B15D9234B5B6A7C2B09D8B6F8C0310E
:1022E000B3F5167F04D2D6F8BC31B3F5FA7F19D313
:1022F00096F8C2310133DBB2642B86F8C23128D89C
:10230000194D95F87130002423B90CE095F871301F
:10231000A34208DD02F03AFE95F86530834204F1ED
:102320000104F3D170BD72B602F038FE0D48B6F864
:10233000BA11426A0D4BA6F8B42101310022426263
:102340005A62D9621A61DA6842F00102DA6062B652
:1023500070BD02F023FE0023C6F8BC3170BD00BF83
:10236000D404002000080040000000200054014078
:1023700070B5CE4C94F8B93082B0002B00F0C88014
:1023800094F8C230002B00F01A81C94DB4F8C42172
:10239000B2F5836F80F0D081A2F130039BB2B3F528
:1023A0007A7F11D294F8B81095F86760C1F10100F6
:1023B000864200F08C8395F872105B009BB2C1F1ED
:1023C0002F010B44A4F8C6312F2A00F2A680002367
:1023D00094F8CB21A4F8C63184F8CA3195F873304B
:1023E0009A4200F2A18094F8BA60002E00F0BF80FB
:1023F000B4F8C6011D2800F285810023A4F8CC3171
:1024000095F8203003EB8303B0EB830F4FEA830191
:1024100080F2848194F8C931002B40F0448194F813
:10242000BA102E22502313FB0123B4F8CC2193427F
:1024300080F28D8094F8D831002B00F02F8194F831
:10244000C331002B00F05C8394F8BA30002B00F00D
:10245000A382EB89B4F8CC014FF4FA6200922833DE
:1024600040F2FF728921FFF751FBA4F8DC0194F8D8
:10247000BF3094F8BA10002B40F00781B4F8CC615B
:1024800084F89F3150222E2312FB0133B3425EDACF
:102490002E2E40F2158294F8BC201E23D340D4F88F
:1024A000BC21934240F20C82B4F8DC31AA899342F9
:1024B0003CBFA4F8DC211346EA8C9A423CBFA4F846
:1024C000DC211346B5F876209A4294F8C13038BF23
:1024D000A4F8DC213BB1B5F97830B4F8DC219A429C
:1024E000C8BFA4F8DC31D4F8E85100212846FFF732
:1024F0006DF8002800F0D7802F2E40F2D4802846B7
:10250000FFF794F8B4F8DC311844A4F8DC01CAE011
:10251000B4F8C431664DA4F8C63194F8CB2195F8CF
:1025200073309A427FF65FAFAB79002B3FF45BAF1D
:1025300003F08AF902F032FD00226623A4F8CC21D0
:1025400084F8CB3194F8C931002B40F0AC8094F87A
:10255000DE31002B00F0B780013B042B00F2B0808D
:10256000DFE813F0AC003B0238023502AC0094F80F
:10257000CE31002B00F0DB8094F8C530002B40F00A
:102580005981D4F8D4614B493046FFF71FF8002831
:1025900040F0F2813046FFF749F8A4F8CC014649F3
:1025A0003046FEF7F5FF00283FF434AF94F8C93108
:1025B0003022A4F8CC21002B3FF43CAF73E094F818
:1025C000BF203B4DB4F8C401002A00F0EF802E7FFD
:1025D000760006F57A7188421DDD94F8B86095F8AA
:1025E0006720B24200F01B8294F89F31002B40F02C
:1025F0001B81002384F8C83140F2FF7300934FF42D
:10260000FA622F23FFF782FA2E7F0346B4F8C40143
:10261000A4F8C6317600C6F57A72824222DD94F8BB
:10262000B83095F86760C3F101018E4200F0258251
:1026300094F89F31002B40F0F7802F230021009366
:1026400040F2FF7384F8C811FFF760FA2E7F03464B
:102650007600B4F8C401A4F8C631C6F57A7398427E
:10266000C0F2E28006F57A76B04200F3DD8094F89D
:102670009F210023A4F8C631002A00F0D580012252
:1026800084F89F3184F8C821CEE02E22502313FB1A
:102690000123B4F8CC219342BFF659AF94F89F615F
:1026A000002E00F0088102B070BD00BFD4040020ED
:1026B0000000002000E0FF440000404201F042FC26
:1026C000002384F8DE312B79002B4BD194F8C32101
:1026D000A4F8DC31002A40F0F88094F8BB30C4F84C
:1026E000BC21012185F86910002B40F0EC8094F8A2
:1026F0009F31002B00F0378294F8BF30002B40F060
:10270000ED80D0E71E283FF47BAE95F8202002EB49
:102710008202920090421146C0F2C18040F2FF72E4
:102720000092A023FFF7F2F9A4F8CC0172E6B4F806
:10273000C631A4F8CC316DE694F8B83095F867103E
:10274000994200F0AB8195F87200A2F583614900CF
:1027500089B2C0F12F00A2F1300301449BB2A4F86A
:10276000C6111CE694F8C331002B40F0CE8094F8DB
:10277000BB20C4F8BC31012685F8696084F89D311E
:10278000002A00F0C08094F8BA00002840F0BF8012
:1027900095F8213003F2DE335B00A4F8E03102F05B
:1027A000AFFF94F8BA0084F89F61B2E02A7F52002C
:1027B00002F57A71884240F3E48094F8B83095F8D5
:1027C00067209A4200F00C8140F2FF7300934FF4AF
:1027D000FA622F23FFF79AF92B7F02465B00B4F8C9
:1027E000C401A4F8C621C3F57A72824240F3E9809D
:1027F00094F8B83095F86760C3F101018E4200F09B
:1028000020812F230093002140F2FF73FFF77EF910
:102810002B7F02465B00B4F8C401A4F8C621C3F5BF
:102820007A72904280F2CD8094F8C230002B3FF44F
:1028300074AEABE5D5E90D322F210092B4F8C60194
:1028400040F2FF72FFF762F9B4F8C6112A7DCC4B53
:10285000A4F8D0012E2980B24FEA5202B3FBF0F067
:10286000B0FBF2F0A4F8D20140F2A480D4F8D46115
:10287000C4493046FEF7AAFE002840F05B8130468E
:10288000FEF7D4FEA4F8CC01BF493046FEF780FE27
:1028900000283FF4BFAD3023A4F8CC31BAE5A02323
:1028A00000931E212F23FFF731F90346A4F8CC3102
:1028B000B4F8C601A4E5B4F8CC612E2E3FF6EBAD1A
:1028C000B4F8DC31FEE503F009F994F8BF30002BD1
:1028D0003FF4E4AE94F89F31002BECD0B4F8C4116F
:1028E0004FF47A70FFF732F92A8900F57A739BB2B8
:1028F000013A9342A4F8E031C0F23E8103F0EEF8D1
:1029000094F89F61CCE602F09FFF94F8BA0094F827
:102910009F6195F86830013BC3EB0312B5F8743042
:1029200003EB82031AB2B2F5B47F9BB2A6BFA3F544
:10293000B4739BB2A4F8E22103F1770212B2A8BFEC
:10294000A4F8E231B2F5B47FA8BFA3F1F102A4F874
:10295000E42103F1EF0212B2B2F5B47FA6BF793BD6
:10296000A4F8E631A4F8E6210023012808BF84F882
:10297000C901A4F8DC3193E640F2FF73A4F8CC312E
:102980000DE6C2F57A729042FFF632AF0023A4F84A
:10299000C63184F8CA3147E74FF4FA62EB89B4F8DC
:1029A000CC0100922F2140F2FF72FFF7AFF8A4F89C
:1029B000DC015CE50023A4F8CC61EE63C4F8D431FB
:1029C000C0E503F57A738342FFF62EAFDEE701F030
:1029D0004BFA75E601F016FB72E601F0E3FA6FE6DA
:1029E000688EEA6E904280F0AA80B4F8C021C72AAF
:1029F00000F2A580C3F101030026012285F86730AB
:102A0000C4F8BC6185F8692002F0C8FA297FB4F8DF
:102A1000C40184F8CA61490001F57A71D4E694F8DA
:102A2000C861A4F8C6314FF0010C84F89FC1002E94
:102A30003FF4FAAEACEB020284F89F3185F86720D0
:102A4000D7E5688EE96E884280F08380B4F8C011C3
:102A5000C7297ED80122002685F86920C4F8BC6108
:102A600085F8673002F09AFA2A7FB4F8C40184F836
:102A7000CA615200C2F57A72C3E694F8C8610021B7
:102A80004FF0010CA4F8C61184F89FC1002E3FF44A
:102A9000CBAE85F8673084F89F11CEE5698EEA6E7B
:102AA000914240D2B4F8C021C72A3CD80122C3F1D8
:102AB0000103002685F8692085F86730C4F8BC61F9
:102AC00002F06CFAB4F8C42184F8CA613BE66A8E5D
:102AD000EB6E9A4220D2B4F8C031C72B1CD8012328
:102AE000002685F86930C4F8BC6185F8671002F0EB
:102AF00055FAB4F8C42184F8CA61A2F130035AE44B
:102B000002F0A2FE95F8693083B3AB89A4F8DA31FC
:102B1000012284F8C32197E494F8C931002BDED157
:102B2000A4F8C43153E494F8C921002ABED1A4F812
:102B3000C4214CE440F2FF73A4F8CC31A4E694F82D
:102B4000C921002A7FF456AF4FF47A70A4F8C4016B
:102B50003AE694F8C91100297FF47CAF4FF47A70FB
:102B6000A4F8C4014DE602F06FFEAEE694F8C3315E
:102B700063B102F01FFAC8E702F0C2FD8EE500BFA4
:102B80000087930300E0FF4400004042FFF708FB8A
:102B9000054B42F2107141F28832E9665A62012314
:102BA00084F8C331E5E700BF0008004010B50E4CC3
:102BB00094F8EC31012B0DD0022B03D0BDE810406E
:102BC000FFF7D6BBB4F8F001FEF736FF002384F818
:102BD000EC3110BDFEF784FD002384F8EC31BDE834
:102BE0001040FFF7C5BB00BFD4040020F8B54F4E1E
:102BF0004F4F96F86710002977D1B7F8E2310133CB
:102C00001AB2B7F8E4310133B2F5B47F1BB2B2BFE8
:102C1000A7F8E221A7F8E2110A46B3F5B47FA8BFEE
:102C20000023A7F8E431B7F8E63101331BB2B3F55E
:102C3000B47F77DAA7F8E63106EB4202B6F84C1318
:102C4000B2F97C3030893B4D3B4C0B4400FB03F325
:102C500085FB0312D81796F82C30C0EBE21003FB6B
:102C600000F0C31784FB0020C3EBA00080B202F089
:102C7000A9FCB7F9E431B6F84C0306EB4303B3F90A
:102C80007C2096F82C300244308900FB02F285FB50
:102C90000201D017C0EBE11003FB00F084FB00231E
:102CA000C017C0EBA30080B202F092FCB7F9E62196
:102CB000B6F84C0306EB4202B2F97C3096F82C20B1
:102CC0000344308900FB03F385FB0315D817C0EBE1
:102CD000E51002FB00F084FB0034C017C0EBA40039
:102CE00080B2BDE8F84002F079BCB7F8E221B7F84D
:102CF000E431013A12B2013B1BB2002AB8BF40F2E4
:102D00006712002BB8BF40F26713A7F8E431B7F899
:102D1000E631A7F8E221013B1BB2002BB8BF40F21D
:102D2000671387E70023A7F8E63185E70000002056
:102D3000D4040020D34D62106766666638B5234D13
:102D40002349EA6E4B6A234C02EB420212FA83F2E9
:102D5000A4F8B43100234B6253095B009BB2A4F882
:102D6000B831C3EBD2039BB29208D4F8BC01EA6637
:102D7000A4F8BA3101E0042802D94A6A9A42FAD387
:102D8000FFF70EFAD4F8BC3194F8BC0094F8BF10E9
:102D90000022013384F89C2184F89D2150EA01022D
:102DA000C4F8BC3105D1EA6E40F213539A4206D9F9
:102DB00038BD132BFCD9EB6EB3F5FA6FF8D80023AE
:102DC00085F86930BDE8384002F0F4B80000002012
:102DD00000080040D4040020F8B5BE4CB4F8F61149
:102DE000B4F8F401B4F8F82194F8D831B4F8DC510F
:102DF000A4F8C0510131A4F8F61194F8FA11013089
:102E000001320B43A4F8F401A4F8F8213ED194F860
:102E1000FB21002A3AD0B4F8C651002D40F0A18120
:102E2000B4F8FC3101339BB244F620618B42A4F824
:102E3000FC312BD9B4F8FE311E2B40F2C78194F837
:102E4000BE30012184F8D811002B00F0C481B4F801
:102E50000012A1484B08A0FB0323DB09B1F5B97FA1
:102E600084F8FA310DD39D4F4AF6AA2601F034F8C2
:102E70006420FEF77BFE94F8FA313E600135AB42E8
:102E8000F4DC94F8C3300BB984F8BF3094F8BD304B
:102E900073B1934AB4F8023292F84E2301339BB2D5
:102EA00002EB8202B3EB820FA4F8023200F3B78088
:102EB00094F8C931002B38D1894D95F8693023B188
:102EC00094F8C331002B40F03281B4F8F831142B60
:102ED00031D895F8A833002B40F0A880B4F8C01181
:102EE00094F8D83123B194F8C331002B40F00E810F
:102EF00094F89F316889002B00F0BF802B89B4F8CB
:102F0000E0215D1C774B00FB02F283FB023CD317F0
:102F1000A3EBEC132B449BB2A4F80832724AA4F83A
:102F2000DA11C2E90D33D062D363B4F80A32013347
:102F3000A4F80A32F8BD94F8C1300022A4F8F821B0
:102F400023B194F8C331002B40F0198194F8BC30C0
:102F5000002B40F09C8094F8CE31002BB9D094F82F
:102F6000C331002BB5D0B4F800226B8A5F48B4F8A7
:102F7000D0615F4F02FB03F3A0FB03235B09C6EBA9
:102F8000C620B0FBF3F0FEF761FA2B7DD4F8F01108
:102F90005B0801FB03F33246564991FBF3F1064609
:102FA0005548FEF751FEFEF751FA3146FEF79AF901
:102FB00039460646FEF70AFB38B9504F30463946C7
:102FC000FEF7E6FA002800F00D81C4F8D471D4F8B9
:102FD000BC31632B3FF67DAF95F8A8330022EA643D
:102FE000002B3FF47BAFB4F8DA3101210A4685F8B3
:102FF000A9138C46B4F8C011C81A90422EDC581A96
:10300000904240F3B580A3EB0C0399B2EA79A4F89F
:10301000C011002385F8AA3385F8702060E70122EB
:10302000002384F80422A4F8023241E7D4F8BC312A
:10303000952BB4F8DA31D8D9952BD6D9D4F8A0216C
:10304000B2F5FA7F8CBF042110210A4685F8A91336
:103050008C46B4F8C011C81A9042D0DDEA6E6344C1
:1030600099B2B2F5FA7FA4F8C0117DD9EB7985F851
:103070007030012285F8AA2332E71A4A00FB01F3D7
:10308000A2FB0323C3F3CF13A4F8083246E794F856
:10309000C331002B3FF41DAFB5F87C23E96E18480F
:1030A000184FFEF7A5FD1849FEF762F8D4F8E811AD
:1030B000FEF718F939460646FEF788FA38B90027B0
:1030C00039463046FEF76EFA002800F08880C4F8D2
:1030D000E87140E7D4040020B9D31FB100300040AC
:1030E00000000020D34D6210002C01401F85EB51E1
:1030F00000E0FF44008793033C00002000004042B2
:10310000800300200000164317B7D138B4F8CC3143
:103110002F2B7FF6EDAE6889344A00FB01F3A2FB4A
:103120000323DB0901339BB2A4F80832F6E601F071
:1031300035FFFFF711F894F8A431002B7FF4C5AEEA
:1031400095F8653094F89C21002B39D095F84F33D1
:103150009A427FF6BAAE012384F8A431FFF7EEFD60
:10316000B3E6A4F8FC3191E6002385F8AA33B7E66C
:10317000EA7985F87020002385F8AA33B0E66B8DD4
:10318000B4F906121A48642203FB02F2FEF730FD7E
:103190001849FDF7EDFFFEF723FAB5F87830E98915
:1031A0001B1A1BB21A468B42A5F878306B89BCBF3C
:1031B0000AB2A5F878209342B8BFA5F87830C5E6E2
:1031C00095F850339A427FF680AEC4E784F8FB51FD
:1031D000A4F8FC515AE6042384F8DE3151E6C4F821
:1031E000E861B8E6C4F8D461F1E600BFD34D6210DF
:1031F0005403002017B7D1382DE9F04F85B002F005
:1032000041F84FF47063CC4AD3F8E010914205D1F5
:10321000CA4AD3F8E410914200F07983C84DC94CF2
:1032200002F06CF902F0F0F9FEF74AFDE378022BA8
:1032300002D12379102B0CD00222C34BE270102252
:10324000227107CBC14EC4F805007160B260FEF771
:1032500011FF94F8B8302A7929896981013B18BF98
:10326000012385F867300AB984F8BA2094F8BF3092
:10327000B3B1E889298AAA89002301264FF47A7715
:10328000323032313232AF84E881298284F8B96039
:1032900085F82D6084F8BA306B712B71AB71AA81FF
:1032A0000522002384F8DE21A4F8FE3102F052F852
:1032B000A74B4AF6AA221A6001F060FF94F8C530C5
:1032C00013B1012384F8CE3101F0D4FFA04FDFF811
:1032D00084B2DFF88492DFF884824AF6AA26B4F832
:1032E000AA11B4F8A831B4F8AC21B4F8AE010B447B
:1032F0001344B4F8B011B4F8B2213E6003440B4457
:10330000134404336A795B10C4F8F031002A40F0AA
:10331000A881B4F80A3242F21072934209D994F8A3
:10332000D811002940F0DA8249F64042934200F277
:10333000FA82B4F8F42144F620639A421BD9B4F916
:1033400006A25046FEF782F85946FDF711FFD4F861
:103350000C12FDF7C7FF99F80030C4F80C02022BDD
:1033600000F07382032B00F06182012B00F0548285
:103370000023A4F8F431D4F8BC21B2F57A7F40F2EE
:103380002A810021B4F8C63184F8CB11C72B40F252
:10339000E48194F8BA1011B19F2B40F2298194F87E
:1033A0001112002900F0C080B3F5C87FC0F027815A
:1033B000D4F8F03194F89E0188FB03C1A1EBE371CE
:1033C000C4F8A01110B10A2A00F2F68194F819325B
:1033D000002B00F08580EB6E322B40F28180604B39
:1033E0001022002183F8101383F81A2383F8462350
:1033F00094F80432002B40F0818094F81C320133A1
:10340000DBB2C82B84F81C3200F2488194F8C93131
:103410004FF0000A84F8C2A1002B40F0A98094F874
:10342000C331504AD4F8F0114F4892FBF1F213FB2C
:1034300002F39BB2A0FB032095F82D20A4F81A32CA
:10344000C008A4F82A02002A40F0988194F81002DB
:1034500095F828104FF4FA638842A5F8763000F208
:103460009E81D4F8BC31632B00F20581EB6EB3F57D
:10347000FA7F40F200810C2385F871301723009306
:103480004FF4FA620D23B4F8C0016421FEF73EFB4D
:10349000364A526A84F8B6014AF6C8739A427FF6F1
:1034A0001EAF94F8C3A1BAF1010F7FF418AF94F8DE
:1034B000CB31013384F8CB3101F070FDB4F8CC315D
:1034C00085F869A02F2B05D8002384F8C33141F279
:1034D0008833EB660023C4F8BC31FFF72FFCFEE60F
:1034E0001F4B0022102183F8101383F81A2383F84E
:1034F000462394F80432002B3FF47FAFD4F80C023B
:10350000FEF794F8B4F81A12B4F80622009183B2C8
:10351000B4F8001294F8100202F036FB02F026FB19
:10352000002384F8043268E7952B94BF64230A23B0
:1035300085F873303CE700BFDAE32559D963B84E0C
:1035400000000020D4040020B8610008D904002045
:1035500000300040610B363B28040020565555557D
:1035600000E100E0C0270900CDCCCCCC0008004031
:10357000B4F8CC31302B4AD994F8D821002A46D05F
:10358000313B572B00F26F8194F82C32002B40F026
:10359000FB81FFF72BFB95F814E0B4F8CC017822FF
:1035A000302141F6583340F22A3CB3FBFEF3BCFB1A
:1035B000FEFCCDF800C0FEF7A9FAA5F8B00380B272
:1035C000FEF7CAFAB5F8B0234FF41673B3FBF2F363
:1035D000A4F81A3283E6B4F8C631A3B9642A84F891
:1035E000CB3100F2BA8094F8BA1000293FF4D7AE7C
:1035F000002184F8CB1194F81112002994D00023F3
:1036000084F8CB31D4E6642A7FF6C3AEBEE694F8E4
:10361000BB304FF0010A84F82CA2002B00F0A780E9
:103620002B8995F82110A3F1130202EB410269895D
:1036300092B2A4F8C02101FB02F2B2FBF3F25344B0
:103640009B1AA4F8083202F05BF8B4F80822C34BC6
:1036500084F89FA1C3E90D22DA630023A4F81A328B
:103660003DE62B890093E86E5B08C8226021FEF7D7
:103670004DFA68814DE60C230093D4F8A001032392
:103680004FF4FA726421FEF741FAEB6E85F871008F
:10369000312B9CBF022385F87130EFE601F0DCFA94
:1036A0000121AF4800F034FEB4F81E0201F070FBB7
:1036B000B4F82222AB4BA4F8200240F6E44A0AFBFD
:1036C00002F2A3FB0213D21A03EB5203B5F8AC23A8
:1036D000A54984F81002DB0A02FB03F3B4F80022C8
:1036E000A1FB0313C2EBC20202EB5313DB10A4F8DD
:1036F0000032FEF707FD9D4BC4F824020AFB00FAD6
:10370000A3FB0A3A4AF30F2ABAF1000FBCBF002309
:10371000A4F8063294F8BE30A8BFA4F806A21BB3E2
:1037200094F8FA31E98BB4F8002201FB03F39A42D2
:1037300017DAB4F8282294F8C9318D48013244F6DA
:10374000206192B200FB03118A42A4F8282200F300
:103750002C81002284F81C225AE6002184F8CB1127
:1037600017E60023A4F8283294F8C931F1E77B4A20
:10377000C2E90D33D36302F067F86EE7B5F8AE33F4
:103780000093E98DAB8C2A8EFEF7C0F995F82810CE
:10379000A5F8760094F8100288427FF662AEB5F87C
:1037A000AE33012200925B0801F10A020A39FEF7EA
:1037B000ADF9A5F8760054E6D4F81402FEF7C6F980
:1037C000D4F8A031B0EB530F1BD9B3F5FA6F18D270
:1037D00094F81822013284F8182294F8B9200021B4
:1037E000C4F8BC119AB9B4F8CC212F2A0FD9002201
:1037F00084F8C321AA895208A4F8DA21012285F8A5
:103800006920002284F89E21C4F81432DEE5EA6EB5
:10381000B2F57A7FEED9EAE794F81032554A43F4CC
:1038200000731380022389F80030A1E5B4F8003258
:103830004D49504AA1FB0313C3F3C70343F480630C
:103840001380012389F8003092E5474A5FFA8AF332
:10385000A2FB03231B09474A43F4C06313800323DD
:1038600089F8003084E5012384F82C32FFF7BEF993
:10387000B4F8CC31C82B04D95023A4F8E2A1A5F8A0
:10388000B033B5F8B003FEF767F9B4F9E231002BB5
:103890007FF425AD384984F8C931012284F89F317D
:1038A00042F22833EB66C4F8A031C4F8143285F82C
:1038B00069204B6294F8BC3084F8C32195F8B22398
:1038C00085F868201422C4F8BC2113B12B8AA4F80F
:1038D000DA31FEF765FC01F087FE00E501F0B4FF88
:1038E0001E4B0025C3E90D55DD6384F8D851A4F8BB
:1038F000CC5184F8FB51A4F8FE5101F07DFE1F4825
:103900004FF48072294602F023FCFEF75FF993F82A
:10391000EC301B4D2B2B5CD0352B57D01F2B04BF0D
:10392000184B2B607BE4039101F08EFF03990B4B46
:1039300084F8D811C3E90D11D963A4F8CC1184F827
:10394000FB11A4F8FE11039101F056FE03990B48F8
:103950004FF4807202F0FCFBD7E700BF002C01405F
:1039600000240140010110001F85EB51FF04EC4FC2
:103970007CFCFFFF2A0400200008004060070020B4
:1039800000000020007C0008134AD36823F00103E4
:10399000D36001F003FB114BC3E90DAAC3F83CA0AF
:1039A00002F0DAF884F82CA2F3E54FF0000AA4F84C
:1039B000CCA101F049FF01F0F1FA94F8C93184F883
:1039C000C3A1A4F8FEA184F8D8A1C2E6044B2B60E1
:1039D00025E4044B2B6022E400540140002C0140FC
:1039E00000F8000800F80108F0B5604CD4E90002C6
:1039F000101A6FF4487240F2765382189A4283B0DC
:103A00002AD85B4E5B4D002333802B78002B3CD0B3
:103A10006B780146ABB9AB78002B00F08E80A8889C
:103A2000554F01333988AB70FEF790F8322866D9CC
:103A300000223B882A706A78AB804AB1D4E9003111
:103A4000C91A40F2E14399424DD9AB794B2B77D853
:103A50000023A868338004E04649484B8868002268
:103A60001A804749474A0B881268A0EB030C94451B
:103A700003DD13440B8003B0F0BD1C1AA242BABF91
:103A80009B1A0B80088003B0F0BD3F4A147874B1D4
:103A90003E4A128890421AD83D494FF47A740988F8
:103AA0000094FEF733F8A86000233380D9E7324B47
:103AB0001A88374B198840F2FF7300932F23FEF7C3
:103AC00025F83028CEBFA860AC602046ECE72A4B32
:103AD000511C1A884FF4FA63009340F2E933FEF761
:103AE00015F8A860E0E72A48AB790288C2EBC20269
:103AF00001331144DBB2C908AB710180A6E73B88F2
:103B00006268C3EBC3012368D31AAA780B44C3F3DA
:103B1000CF03322A3B808ED9193B9BB23B80A3F264
:103B2000D6631C4A03EBD3735B1082F82130012368
:103B30006B7000F007FA3B887DE780B2A8806FE7E2
:103B4000134A1449138819339BB21380A3F2EE234E
:103B500003EBD3735B10002481F820302C70FEF748
:103B600089FAAC7100F01EFA72E700BF600700200E
:103B7000DE0600203407002018000020D2060020B6
:103B800098060020C80300208D0500201A000020A0
:103B900016000020D40400201A4A9388591E0229D6
:103BA00030B413D8184BD9683B290DD80121174DD3
:103BB0001748197400232B70164C174B21700E25D3
:103BC000057020209071197030BC7047043B042BA5
:103BD000FAD80D4BD9686329F6D80D480D4D0B4C1A
:103BE0004FF0030C83F810C00B4B4FF0070C012172
:103BF00080F800C02020297021709071197030BCAD
:103C0000704700BFC803002034070020D203002003
:103C1000D303002096050020CF060020F8B5284BDE
:103C2000284F1968002544F6206E1A46A7F804E0CC
:103C300003F17804AC462E4652F8043F8B42A3EBC6
:103C40000100194606D070453CBF1FFA80FE0126D0
:103C500084440125A242EFD10EB1A7F804E00DB1D2
:103C60004FEA5C15184C194A2378D560012B23D0F4
:103C7000174D2B78012B15D02278134311D1FFF764
:103C80008BFFBB88C93B44F656529BB2934208D87F
:103C900001231049104A2B708F2008700221B9713E
:103CA0001370F8BDBA88C93A44F6565192B28A42A6
:103CB000F7D80849084AEFE7FFF76EFFD8E700BFDB
:103CC00060070020C803002096050020340700206C
:103CD00097050020D2030020CF06002070B5504C7D
:103CE000237813B14F4B1B7833B94F4B1B78002B04
:103CF0004FD0012B0AD070BD4C4B1B78002B35D018
:103D000001F03CFA4A4B02221A7070BD454B1B78F9
:103D1000002B31D1474D2B78012B6FD0464B1B78B0
:103D2000012B62D02378002BE5D12B78002B3AD0E1
:103D30004249434B4A7C072A36D81888052833D98C
:103D4000404C4D69E06F24680132D2B22844001B18
:103D5000082A4A74486127D1C0F3CF023A4CC0F315
:103D6000CF101518101A258108831DE001F028FADC
:103D70002F4B01221A7070BD2C4B1B787BB1334B3B
:103D80001888FDF759FEFDF7ABFCBDE8704001F067
:103D9000F5B9FFF743FFBDE8704001F0EFB9BDE8AA
:103DA000704001F00DBA264B294C208830B9234AC7
:103DB000127842BB1A8801321A8070BD40F2DC5280
:103DC000002690421E8096D91C4D698BFDF7BEFEE1
:103DD00032281ED82B7F0133DBB2322B2B7701D94F
:103DE0006E7896B123886B8370BD01F03BFA164B59
:103DF00088B103229A7101F0C1F993E7FDF770FCD5
:103E000001F0BCF98AE7188070BD00F0FBF80123CF
:103E10002B702E77E6E702229A71FFF7E5FDEAE7BD
:103E2000AC060020ED060020CF0600205C07002035
:103E3000C0060020960500209705002034070020CA
:103E4000D206002060070020C8030020C40600201E
:103E50009A0600200B28034B28BF0B204000187047
:103E6000704700BF5107002070B5164C41F27073C7
:103E7000E36272B6144D154B3C224AF6AA262E6018
:103E8000A2621B78E363C4E90D33012001F01AFD3F
:103E90004B20FDF76BFE5023A3624B20FDF766FE1F
:103EA0005A23A3624B202E60FDF760FE01F0CCFC8C
:103EB000074A084912880023A3620B80E26262B6B7
:103EC00070BD00BF002C01400030004051070020B1
:103ED00008000020DE06002010B572B6144C154A0A
:103EE000154B4AF6AA2141F27070E062116050222F
:103EF000A2621B78E363C4E90D33032001F0E2FC06
:103F00006420FDF733FE4623A3626420FDF72EFEF6
:103F10002823A3626420FDF729FE01F095FC074ADF
:103F2000074912880023A3620B80E26262B610BDCB
:103F3000002C014000300040510700200800002004
:103F4000DE06002010B5124C124B41F27071322285
:103F5000E162A2621B78E363C4E90D33022001F041
:103F6000B1FC9620FDF702FE0B4A4AF6AA211E2359
:103F700011609620A362FDF7F9FD01F065FC074A88
:103F8000074912880023A3620B80E26210BD00BFC4
:103F9000002C0140510700200030004008000020A4
:103FA000DE06002010B5124C124B41F2707128222F
:103FB000E162A2621B78E363C4E90D33022001F0E1
:103FC00081FC9620FDF7D2FD0B4A4AF6AA21502328
:103FD00011609620A362FDF7C9FD01F035FC074A88
:103FE000074912880023A3620B80E26210BD00BF64
:103FF000002C014051070020003000400800002044
:10400000DE0600202DE9F041154D41F27073EB62A0
:1040100072B6144BDFF850801B78144FEB63C5E980
:104020000D3377244AF6AA26A7FB04300009C8F806
:10403000006001F047FC63100A33AB620A20023CC7
:10404000FDF794FD631CEFD101F0FEFB084A09491E
:1040500012880023AB620B80EA6262B6BDE8F08191
:10406000002C01405107002000300040CDCCCCCCCA
:1040700008000020DE060020002103E00B4B5B5807
:10408000435004310A480B4B42189A42F6D30A4A6D
:1040900002E0002342F8043B084B9A42F9D301F0B6
:1040A0001FFE02F031F8FFF7A7F87047D86100084B
:1040B00000000020DC030020DC0300208408002036
:1040C000FEE70000836861F300038360704700BF70
:1040D00000230122037043708370C270704700BFD9
:1040E00043680A7862F30823436083684A7862F37E
:1040F0004103836083688A7862F3CB238360CB7843
:10410000C26A013B63F31752C2627047836861F36E
:1041100008238360704700BF836843F0080383600F
:10412000704700BF8068C0F3C0007047836843F0E9
:1041300004038360704700BF8068C0F3800070474D
:1041400010B4112917D8DFE811F0120079007E00B1
:10415000830088008D00920097009C00A100A600BB
:10416000AB00B000B500BA00BF00C4007400046921
:1041700063F302040461013A0F2A0DD8DFE802F06C
:104180000E13181D22272C31363B40454A4F540848
:10419000C36A61F3D333C36210BC7047436B61F3EE
:1041A00004034363F8E7436B61F349134363F3E7A5
:1041B000436B61F38E234363EEE7436B61F3D333C9
:1041C0004363E9E7436B61F318534363E4E7436BED
:1041D00061F35D634363DFE7036B61F30403036330
:1041E000DAE7036B61F349130363D5E7036B61F30C
:1041F0008E230363D0E7036B61F3D3330363CBE711
:10420000036B61F318530363C6E7036B61F35D63EC
:104210000363C1E7C36A61F30403C362BCE7C36A13
:1042200061F34913C362B7E7C36A61F38E23C362C4
:10423000B2E7C46863F35754C4609CE7046963F34E
:10424000C504046197E7046963F38814046192E785
:10425000046963F34B2404618DE7046963F30E344E
:10426000046188E7046963F3D134046183E7046976
:1042700063F3944404617EE7046963F35754046173
:1042800079E7046963F31A64046174E7046963F30A
:10429000DD6404616FE7C46863F30204C4606AE725
:1042A000C46863F3C504C46065E7C46863F3881435
:1042B000C46060E7C46863F34B24C4605BE7C46810
:1042C00063F30E34C46056E7C46863F3D134C4604A
:1042D00051E7C46863F39444C4604CE783680729DA
:1042E0008CBF43F000736FF359638360836861F39D
:1042F00053438360836862F314538360704700BF45
:10430000024B9A6860F3D7529A60704700240140CC
:10431000836861F396538360704700BF054B1A684A
:1043200018B961F300021A60704761F310421A6015
:10433000704700BF0024004010B412490B6843F0DE
:1043400001030B600B689B07FCD54B680D4A6FF3AC
:1043500001034B60536813F00C0FC3F38101F9D1D3
:10436000136823F0867323F48033136041F61074CE
:104370004FF480104FF41F035160D462106310BCDF
:104380009360704700100240030C03F1804303F573
:10439000043300F01F001A68012303FA00F030EA2A
:1043A00002030CBF01200020704700BF030C03F183
:1043B000804303F5043301291A6800F01F0006D07A
:1043C000012101FA00F022EA00001860704701FAAA
:1043D00000F0104318607047030C03F1804303F5AD
:1043E000043301291A6800F01F0006D0012101FAE8
:1043F00000F022EA00001860704701FA00F0104354
:1044000018607047042809D8DFE800F0090F151B71
:1044100003000F4B5A6A61F300025A6270470C4B5B
:104420001A6861F300021A607047094B1A6861F359
:1044300010421A607047064B1A6861F318621A60DE
:104440007047034B1A6A61F300021A62704700BF9B
:1044500000100240024B5A6860F307125A6070471E
:1044600000100240024B5A6860F30A225A607047FB
:1044700000100240024B5A6860F3CD225A60704728
:1044800000100240054B5A6860F38F325A605A6838
:10449000C0F3800060F31C725A6070470010024045
:1044A000134BA0B95A6860F3104284465A60104B0F
:1044B0005A6861F395425A605A68C1F3011060F37B
:1044C0005E725A60DA6A6CF31A62DA6270475A688E
:1044D00042F480325A605A6801280BBF6FF3514290
:1044E00042F400324FF0020C4FF0000C5A60DEE74D
:1044F00000100240024B5A6860F301025A60704794
:1045000000100240024B5868C0F38100704700BFA2
:104510000010024038B53F4D6B6813F00C0F044695
:10452000C3F3810228D0022A2FD03B4B23603948A5
:104530003A4A41683A4DC1F30311515CCB40636084
:104540004168C1F302211144097C23FA01F1E160C1
:104550004168C1F3C221695CCB40A36045684168F2
:10456000C5F30070C1F3813141EA80010A44127E33
:10457000B3FBF2F3236138BD6B6D9805D5D52B6B7A
:104580009901D2D5274B2360D1E76968EB6A002BEC
:10459000C1F300411DDAEA6AEB6AC2F3031CEA6A5E
:1045A000C3F3082302F0070269B369681E4811F4D7
:1045B000003F194908BF08460021A3FB000503FB83
:1045C00001F10CFA02F20023FDF750F803462060D7
:1045D000ADE76B686A6812F0C04FC3F38343C2F360
:1045E00041700CD10F2B0AD0023319B1094A52681D
:1045F00092030AD50C4800FB03F3236097E70133CD
:1046000003EB0013F1E70848D7E7034800FB03F387
:1046100023608CE70010024000127A0088610008D5
:1046200098610008006CDC0200093D00012805D0FB
:10463000054B5A6D6FF305125A657047024A536D68
:1046400043F030035365704700100240016840F2A8
:10465000FF42024000236FF30001B2F5816F016059
:10466000036043608360C3600ED2C3B20A4A0B4941
:10467000083BA2FB03231B0948689B000F2202FA98
:1046800003F303434B607047B2F5916FFBD2C3B2A3
:10469000014A0349083BECE7CDCCCCCC00000240FA
:1046A00000040240036812B119430160704723EA15
:1046B00001010160704700BF036861F300030360FC
:1046C000704700BFB0F1805F8CBF044B044B1B6888
:1046D000034214BF01200020704700BF00040240C5
:1046E000000002400023C0E90033C0E90233038226
:1046F000704700BF03684BF6EF7213400360026817
:104700000B891343036003684A7C62F30D33036033
:104710000368CA7B62F38B23036003688A7B62F3BE
:104720000923036003684A7B62F3C71303600368CD
:104730000A7B62F3861303600A7C036862F3451305
:104740000360D1E9002310B44C894460826010BC3E
:10475000C3607047014BD860704700BF0020024023
:10476000024B0349034A59605A60704700200240D7
:1047700023016745AB89EFCD024A136943F08003FB
:1047800013617047002002401B4A136943F0020383
:1047900013615061136943F040031361D368D90773
:1047A00004D4D3685B0720D5012011E04FF080438B
:1047B000D168C80712D4D168490713D4D268D20689
:1047C00003F1FF334CBF02200320002B08BF04205D
:1047D000094B1A696FF341021A617047013BE7D137
:1047E0000420F5E7013B0120EFE7D36813F0100F39
:1047F00014BF02200320EBE700200240194A13698E
:1048000043F0010313610160D368D90704D4D3686E
:104810005B0720D5012011E04FF48013D168C80751
:1048200012D4D168490713D4D268D20603F1FF33FA
:104830004CBF02200320002B08BF0420094B1A693B
:104840006FF300021A617047013BE7D10420F5E7DE
:10485000013B0120EFE7D36813F0100F14BF0220D3
:104860000320EBE70020024070B58A790B68032A29
:104870001FFA83FE4FD0002A43D091F804C0C979B3
:104880000CF0040C02F008024CEA020201F0030CE6
:1048900042EA0C0C9DB2DBB2B3B100230F2645FAFD
:1048A00003F19A0011F0010F06FA02F403F101037B
:1048B00008D0016821EA0401016001680CFA02F2E3
:1048C0000A430260082BEAD1BEF1FF0F18D94FEA64
:1048D0001E2E00230F254EFA03F19A0011F0010F4E
:1048E00005FA02F403F1010308D0416821EA04014A
:1048F000416041680CFA02F20A434260082BEAD197
:1049000070BD4A79182A02F00F0C9DB207D0282AF0
:1049100008BF4561BFE775464FF0000CBBE7056176
:10492000B9E700BF024B4FF6FF72C0E900237047A2
:1049300000040003C0F30723C0F3074CC3F12003B6
:10494000A3EB0C024FF0FF339340D340020E02F171
:10495000804202F5803210B423FA0CF3146803FA93
:104960000CF324EA030411B9146010BC7047C0B200
:1049700000FA0CF32343136010BC70471F4BDB6835
:10498000C3F3022300B5C3F1070EBEF1040F03F118
:10499000040C28BF4FF0040EBCF1060F21D9033BD5
:1049A0004FF0FF3C0CFA03FC22EA0C024FF0FF3CF4
:1049B0000CFA0EFC21EA0C019940002841EA0201A0
:1049C00012DB0F4A09011318C9B283F8001301233F
:1049D000410900F01F0003FA00F042F821005DF8E1
:1049E00004FB00221346E1E7064B00F00F0009012B
:1049F0000344C9B219765DF804FB00BF00ED00E086
:104A000000E100E0FCEC00E008B5354B98421FD017
:104A1000B0F1804F26D0334B98422FD0324B984282
:104A20000CD0324B984233D0314B98423AD0314B74
:104A3000984241D0304B984248D008BD2F480121C0
:104A4000FFF7CAFCBDE808402C480021FFF7C4BCB2
:104A50002B480121FFF7C0FCBDE808402848002191
:104A6000FFF7BABC01214FF48010FFF7B5FCBDE899
:104A7000084000214FF48010FFF7AEBC214801210F
:104A8000FFF7AAFCBDE808401E480021FFF7A4BCC0
:104A90001D480121FFF7A0FCBDE808401A4800218D
:104AA000FFF79ABC19480121FFF796FCBDE80840C2
:104AB00016480021FFF790BC15480121FFF78CFC38
:104AC000BDE8084012480021FFF786BC11480121CB
:104AD000FFF782FCBDE808400E480021FFF77CBCD0
:104AE000002C01400004004000080040000C004081
:104AF000004C0140005001400054014002001000F1
:104B00000B000C00010010000300100013000C004B
:104B100014000C0015000C00036861F3C713036058
:104B2000704700BF062909D8DFE801F013080E0816
:104B300009080400C36962F3CB23C3617047C369EA
:104B400062F3C303C3617047836962F3CB2383615C
:104B50007047836962F3C30383617047062909D8EC
:104B6000DFE801F0090E13181D220400036A62F346
:104B70000C3303627047036A62F3000303627047F9
:104B8000036A62F3820303627047036A62F30413E9
:104B900003627047036A62F3861303627047036A15
:104BA00062F3082303627047036A62F38A23036295
:104BB000704700BF2DE9F04186B0054601A81746B1
:104BC0001E468846FFF7A6FCDDE90334114A9542EC
:104BD00008BF1C4604EB84046400B4FBF8F10E4CDF
:104BE000A4FB0134E40804EB8403A1EB4301042992
:104BF000AB6888BF0134A4B264F30F03AB60EB6809
:104C000067F30C33EB602B6966F30D332B6106B051
:104C1000BDE8F08100380140CDCCCCCCC36861F355
:104C20004D33C360704700BFC36861F3C303C36003
:104C3000704700BFC36861F38203C360704700BF61
:104C4000436961F3C7134361704700BF436961F370
:104C5000C3034361704700BF064B0748B3F804C065
:104C60000649074AA0F800C018885B8808801380AE
:104C7000704700BF54070020F2060020F60600200F
:104C80006C06002030B5012187B04FF4A010FFF76B
:104C90008DFB002202210B20FFF770FE3648374CB7
:104CA000FFF7D4FC01A8FFF71DFD354B354A32480C
:104CB000019301A940F201234FF44035ADF81430BF
:104CC000CDE902450492FFF715FD01222A48022191
:104CD000FFF7E8FC28480121FFF7EEFC01212A48F4
:104CE000FFF764FB0220FFF7CDFB6846FFF7F0F902
:104CF00001240325002325488DF8023069468DF8EC
:104D000000408DF801408DF80350FFF7E9F91F4886
:104D10002B4622462946FFF713FA1C482B4606214C
:104D20000222FFF70DFA2B462A4610211748FFF7FB
:104D300007FA2046FFF7E4FA224614480721FFF756
:104D4000CDFA12482146FFF7E1F910482146FFF756
:104D5000B9F90E48FFF7E0F90C48FFF7E3F900282E
:104D6000FAD10A48094CFFF7E1F92046FFF7E4F9C8
:104D70000028FAD107B030BD0800024054070020D7
:104D80004C240140000101010900180000240140E9
:104D900048F2E80300FB03F3002BB8BF03F6FF73F0
:104DA000064A43F23810A0EB233082FB0023C017E1
:104DB000A0EBE300053000B2704700BF310CC330F8
:104DC000704700BFFEE700BFFEE700BFFEE700BF81
:104DD000FEE700BF704700BF704700BF704700BFCD
:104DE000704700BF10B50220FFF76CFC012800D00F
:104DF00010BD054C6060FFF72FFF0820FFF762FC35
:104E0000012808BF606010BD0000024008B54FF4E3
:104E10000050FFF757FC012807D10B4B4FF480528D
:104E20005A605A6C6FF300025A648020FFF74AFC04
:104E3000012800D008BD044B4FF480525A605A6CD0
:104E40006FF300025A6408BD0000024008B54FF439
:104E50008000FFF737FC01280CD04FF40010FFF75B
:104E600031FC012819D04FF40000FFF72BFC01287A
:104E700027D008BD194B1B78002BEED0184A1949D2
:104E8000136A4FF4800043F00203136248604FF44A
:104E90000010FFF717FC0128E5D1124B4FF48012E8
:104EA0005A60DA6E6FF30002DA66FEF717FF0E4BF8
:104EB0004FF400421A614FF40000FFF703FC012891
:104EC000D7D1084B4FF480125A60DA6E6FF30002AC
:104ED000DA66BDE80840FEF701BF00BF9705002075
:104EE000000400400000024000040140044B5A69E5
:104EF000120300D470474FF400225A61FDF7E4B961
:104F0000000401400449054B4FF6FE700022086181
:104F10001A61FDF761BF00BF004C0140002C014049
:104F20000349044A00230B611361FDF78FB900BFE9
:104F300000540140002C0140034B4FF6FE714FF628
:104F4000FD7219611A61704700500140704700BF3F
:104F5000074B1A69910744BF4FF6FD721A61044B63
:104F60001A69D20744BF4FF6FE721A61704700BF3C
:104F700000040040044B5A69120400D470474FF4F7
:104F800000425A61FDF712BE00040140024B18684E
:104F9000C0F38030704700BF00240040044B1A6803
:104FA0004FF4002122F400221A605961704700BFBB
:104FB00000040140024A136843F400231360704761
:104FC000000401401A4A1378012B2CD0042B2AD05C
:104FD000022B23D0052B21D0032B0ED0062B0CD077
:104FE000144B1B7883B1144B9A6822F400229A6008
:104FF000DA6842F40022DA607047104B104A1A60F7
:105000000C4B1B78002BEED10B4B9A6842F400221C
:105010009A60DA6822F40022DA607047074B094987
:1050200019601378D8E7054B074919601378CFE763
:1050300068000020650000200004014000240040BA
:10504000C1000040E1000040D10000402DE9F043E4
:105050000029B4BFCE1C0E4626F00303073383B0ED
:1050600023F0070300AFADEB030DB6106D46884685
:105070008146144600213246284601F069F8B8F10D
:10508000030F17DD4846291F0022837890F803801C
:1050900090F800E090F801C01B0443EA086343EA7B
:1050A0000E03013243EA0C23964241F8043F00F11B
:1050B0000400EADC3E60FFF753FBC4F30903EBB1E5
:1050C00000237B607B683A689A4211D978687B68D4
:1050D00004EB800055F82310FFF790FB0320FFF747
:1050E00039FB7B6801337B607A683B689A42EDD379
:1050F000FFF742FB0C37BD46BDE8F0832046FFF7C3
:1051000043FBDDE7002A09DD431E013103EB020CFE
:10511000081AC25C03F8012F6345FAD1704700BF3B
:1051200070B5114E114C1023042200213046FCF7BB
:1051300037FD0F4B1022D96ED9660025326120460B
:105140006562FFF761FC0B4B0B224121A1612262DA
:105150001A78A2624FF6FF73E3626369064A43F06E
:1051600001036361157070BD000C01400004004034
:1051700000000240D20300205C07002008B5FFF7C2
:10518000CFFF0A4B0A480B490B4A586799671178B9
:105190000A4A1967D16841F40071D160116841F081
:1051A000010140F68B101160D86608BD0000024076
:1051B0003404004060070020CE03002000040040BB
:1051C00070B5204D204CEB6E43F010032046EB668B
:1051D000FFF71AFC602103231C4AA16123621278A5
:1051E0001B4BA2625F210122E1621A7063691949B7
:1051F000194A1A4843F001036361194B6967AA67AA
:105200005A7817322A67E96E41F00201E966E96EC1
:1052100041F00801E966E96E41F00101E966E168E3
:1052200041F40071E160616C41F400416164216806
:1052300041F001012160BDE87040102304220821E3
:10524000FCF7AEBC00000240000400404407002010
:105250005C070020340400403C040020000C0140A6
:10526000D2030020024B986800F01000704700BF86
:10527000000C01400248102318220021FCF790BCCA
:10528000000C014062B670471C4B4FF4AA7210B577
:105290001A60FFF751F801210020FFF7B3F8012051
:1052A000FFF772F801280446F9D100202321FFF707
:1052B000F7F821460220FFF7A5F81920FFF764F858
:1052C00001280446F9D10020FFF7C4F80420FFF7B5
:1052D000D1F80420FFF7C6F82046FFF7A7F902200F
:1052E000FFF708F9FFF70EF90228FBD10020FFF7BE
:1052F0009DF9BDE8104000F033BD00BF0020024022
:1053000010B51048104C0121FFF750F80F4801214B
:10531000FFF74CF82046022304220321FCF740FC4F
:105320002046202304220321FCF73AFC084B0020EE
:1053300083F8460340229A600121BDE81040FEF741
:10534000EDBF00BF020018000008014009001C006A
:1053500000E100E0084B10B44CF6CC4245F2555445
:105360001C6004201A604FF47A614AF6AA22586041
:1053700010BC99601A6070470030004070B5012180
:105380004FF4C010FFF712F82E482F4C2F4D01217B
:10539000FFF70CF82E480121FFF7CCFA6823002113
:1053A00040F6B83046F66802E062A1622046A2618B
:1053B000E3610122FFF7B6FB204601220221FFF73D
:1053C000B1FB012220460421FFF7ACFB204601215E
:1053D000FFF7A2FB636C1F48642262F30703636458
:1053E0000121FEF7E3FF1C480121FEF7DFFF2846FD
:1053F000022304220821FCF7D3FBA4F5105428460D
:10540000012304220821FCF7CBFB20468023042241
:105410000821FCF7C5FB20464FF4806304220821D5
:10542000FCF7BEFB20464FF4007304220821FCF772
:10543000B7FB20464FF48073BDE87040042208217A
:10544000FCF7AEBB0B001800002C0140000C014023
:1054500001040024020018000300180038B51F489A
:105460001F4D0121FEF7A2FF1E480121FEF79EFFFE
:1054700001214FF4C010FEF799FF1B480121FFF7EF
:1054800059FA1A480121FFF755FA01214FF4A010EB
:10549000FEF78CFF2846102304220021FCF780FB36
:1054A0001349144A40F68A101023C86682F8103354
:1054B0004FF480311160104C4FF6FF72E262A3622C
:1054C000226842F080022260002104222846FCF774
:1054D00067FB236843F00103236038BD0300180015
:1054E000000C014001001C000203103002040824DB
:1054F0000000024000E100E00004004070B5FFF74A
:10550000C3FE274C01214FF4A010FEF74FFF1023DC
:1055100084F810334FF480332360FFF72FFF2148C6
:105520000121FEF743FF204B20484A224FF6FF7629
:10553000DE6201219A62FEF739FF1D4B32218F2274
:10554000D9629A62302384F818334FF08073236055
:10555000FFF7D6FE17480121FEF728FF164B4FF440
:10556000FA724B25DA629D621A6842F080021A6074
:10557000002384F81A334FF0806323600F48012121
:10558000FEF714FF0E4BDE629D621A6842F0800245
:105590001A60FFF763FFBDE8704000F027BB00BF53
:1055A00000E100E002001C000008004013001800A9
:1055B000004C014015001800005401401400180070
:1055C00000500140014B5863704700BF002C014060
:1055D000014B9863704700BF002C0140014BD8631A
:1055E000704700BF002C0140024A536943F0010399
:1055F00053617047002C0140024B0022DA625A626C
:10560000704700BF0004004010B5384C012220460E
:105610000021FFF7A3FA204601220221FFF79EFA9C
:10562000204601220421FFF799FA01221146204663
:10563000FFF794FA204601220321FFF78FFA204654
:1056400001220521FFF78AFA2268294B294842F0F6
:1056500001022260626C42F400426264626942F0BC
:10566000010262611968244A41F001011960596917
:1056700041F001015961D96821F00101D960016847
:1056800041F001010160116841F0010111605169AF
:10569000A3F5006341F0010151611A6842F0010273
:1056A0001A605A6942F001025A61DA6842F0010256
:1056B000A4F59434DA60FFF7E5FA012200212046D0
:1056C000FFF74CFA23680D4A43F0010320212360C1
:1056D00082F828134FF48073536002F1C04202F540
:1056E0000C52136843F40043136010BD002C0140BA
:1056F00000540140005001400008004000E100E07B
:1057000070B51A4C1A4D20464FF4806304221021C4
:10571000FCF746FA4FF4806060614FF40073204656
:1057200004221021FCF73CFA4FF4007060614FF442
:105730008073204604221021FCF732FA4FF4807166
:1057400061612846022304220821FCF729FA284631
:10575000012304220821FCF723FA20468023BDE818
:10576000704004220821FCF71BBA00BF000801406A
:10577000000C014010B50E4B1B788BB90D4C01236A
:10578000042210212046FCF70BFA01236361BDE8D7
:10579000104009484FF4007304220821FCF700BAB6
:1057A0000448012304220821FCF7FAF9EFE700BFBF
:1057B00004000020000C01400008014010B50E4B11
:1057C0001B788BB90D4C8023042210212046FCF756
:1057D000E7F980236361BDE8104008484FF4807307
:1057E00004220821FCF7DCB90448802304220821A4
:1057F000FCF7D6F9EFE700BF0400002000080140E5
:1058000010B50E4B1B788BB90D4C022304221021CE
:105810002046FCF7C5F902236361BDE81040094842
:105820004FF4806304220821FCF7BAB9044802232C
:1058300004220821FCF7B4F9EFE700BF04000020C0
:10584000000C01400008014038B51C4D1C4C0223DF
:10585000042210212846FCF7A3F902214FF48063AB
:105860000422696120461021FCF79AF94FF4806107
:1058700001230422616128461021FCF791F90121DE
:105880004FF400730422696120461021FCF788F967
:105890004FF4007080230422102160612046FCF741
:1058A0007FF98023636104224FF480731021204626
:1058B000FCF776F94FF48073636138BD000C01404A
:1058C00000080140013838B5052800F20181DFE801
:1058D00000F02D5781ABD5037E4D7F4C2846012328
:1058E00004221021FCF75CF90121696120464FF484
:1058F000007304221021FCF753F94FF4007060612B
:105900008023204604221021FCF74AF980232361DA
:1059100020464FF4807304221021FCF741F94FF424
:1059200080736361BDE83840FFF76ABF6A4C694D18
:105930002046802304221021FCF732F98020606188
:105940004FF48073204604221021FCF729F94FF40C
:10595000807161612846012304221021FCF720F99F
:1059600001232B6120464FF4007304221021FCF721
:1059700017F94FF400736361BDE83840FFF740BF8B
:10598000544D554C2846022304221021FCF708F9F7
:105990000221696120464FF4806304221021FCF744
:1059A000FFF84FF480616161284601230422102131
:1059B000FCF7F6F801232B6120464FF40073042214
:1059C0001021FCF7EDF84FF400736361BDE8384037
:1059D000FFF7F4BE3F4D404C28460123042210211E
:1059E000FCF7DEF80121696120464FF400730422C0
:1059F0001021FCF7D5F84FF40071616128460223AD
:105A000004221021FCF7CCF802232B6120464FF42E
:105A1000806304221021FCF7C3F84FF480636361B4
:105A2000BDE83840FFF7CABE2B4C2A4D20468023E4
:105A300004221021FCF7B4F8802060614FF48073D9
:105A4000204604221021FCF7ABF84FF4807161610D
:105A50002846022304221021FCF7A2F802232B611E
:105A600020464FF4806304221021FCF799F84FF48C
:105A700080636361BDE83840FFF77CBE154D164C6E
:105A80002846022304221021FCF78AF802216961CA
:105A900020464FF4806304221021FCF781F84FF474
:105AA000806060618023204604221021FCF778F892
:105AB0008023236120464FF4807304221021FCF7D9
:105AC0006FF84FF480736361BDE83840FFF752BE52
:105AD00038BD00BF000C01400008014038B51C4D26
:105AE0001C4C0223042210212846FCF759F80221FD
:105AF0004FF480630422296120461021FCF750F8FE
:105B00004FF4806101230422616128461021FCF7D3
:105B100047F801214FF40073042229612046102127
:105B2000FCF73EF84FF400708023042210216061DE
:105B30002046FCF735F88023236104224FF480735C
:105B400010212046FCF72CF84FF48073636138BDB8
:105B5000000C01400008014008B5FFF751FEFFF7B7
:105B600009FEBDE80840FFF729BE00BF044A054B07
:105B700012789A645A6C42F001025A64704700BF6E
:105B8000D40300200000024010B5174CBDF808C037
:105B90002271120AE2701A0AA1706271090A4FEAB0
:105BA0001C22617084F808C02070A371E271A446C1
:105BB00004F1080E0021414008224B0011F0800F33
:105BC00083F0070314BFD9B2490002F1FF3308BFC5
:105BD000C9B213F0FF02F0D1F44502D01CF8010F56
:105BE000E9E7617210BD00BF6008002030B53148A0
:105BF000314C89B00121FEF7D9FB30480121FEF775
:105C0000D5FB01214FF4A010FEF7D0FB2C4B2D4803
:105C100001A94022CDE90123FEF726FE2046FEF72A
:105C200015FD03A8FEF75EFD274B1A78274BADF84C
:105C300016200025264A049303A920464FF48073BA
:105C40001024ADF8144003920693ADF81C50FEF7F3
:105C500051FD204B204C5A6C204842F002025A64FD
:105C60005A6C42F008025A640121FEF763FE2B468B
:105C70002A4620464FF4E131FEF79CFF20460121E1
:105C8000FEF7D2FF20460121FEF7D4FF2046012176
:105C9000FEF7DCFF20460121FEF7D2FF204601215E
:105CA000FEF7BCFF2A4603210E20FEF767FE09B06F
:105CB00030BD00BF0E001800440002400300180071
:105CC00000040801000C0140D403002060080020FB
:105CD0000438014000000240003801400104102C4B
:105CE00030B41B4A1B49D36943F08053D36191F808
:105CF000503043F0040381F85030D3696FF31C73C4
:105D0000D361136843F00103136013689B07FCD54C
:105D100053680F496FF3010353604B6813F00C0F86
:105D2000C3F38102F9D10B680B480C4C23F0867346
:105D300023F480330B6041F610754FF480134A60F2
:105D4000CD620B634FF41F038B60846030BC7047DF
:105D5000001002400070004000ED00E0001000085C
:105D600010B5FEF7CFFB60B1022816D02C482D4BA2
:105D70002D495B682D4AC3F30313CB5CD8401060F8
:105D800010BD284B5A6D9205F0D51A6B244B28484C
:105D900012F0007F08BF1846E9E7224B5968DA6A1B
:105DA000002AC1F300411CDAD86ADC6ADA6AC0F35F
:105DB000031EC4F3082402F0070259B35B681D48B0
:105DC00013F4003F164B4FF0000108BF18460EFABF
:105DD00002F20023A4FB000E04FB01F1FBF746FCDA
:105DE000C5E758685B6813F0C04FC0F38340C3F346
:105DF00041720BD10F2809D0023019B1094B5B68F1
:105E00009B0309D50B4B03FB00F0B0E7013000EB1F
:105E10000210F2E70748DAE7014B03FB00F0A6E7C0
:105E200000127A0000100240A8610008D803002088
:105E3000006CDC0200093D002DE9F047089E0D468C
:105E400004468846002B4DD18A42944668D9B2FA5E
:105E500082F252B101FA02F3C2F1200120FA01F1FB
:105E60000CFA02FC41EA030894404FEA1C45210C5D
:105E7000B8FBF5FE1FFA8CF705FB1E8341EA0343CE
:105E80000EFB07F199420BD91CEB03030EF1FF3017
:105E900080F01E81994240F21B81AEF1020E6344F4
:105EA0005B1AA4B2B3FBF5F005FB103344EA0344DC
:105EB00000FB07F7A7420AD91CEB040400F1FF33EB
:105EC00080F00881A74240F2058164440238E41B57
:105ED00040EA0E4000211EB1D4400023C6E9004331
:105EE000BDE8F0878B4208D9002E00F0EE8000213B
:105EF000C6E900050846BDE8F087B3FA83F100293A
:105F00004AD1AB4202D3824200F2F980841A65EB97
:105F1000030301209846002EE2D0C6E90048DFE7DF
:105F200002B9FFDEB2FA82F2002A40F09180A1EBC2
:105F30000C054FEA1C471FFA8CFE0121B5FBF7F355
:105F400007FB1350250C45EA00450EFB03F0A84261
:105F500008D91CEB050503F1FF3802D2A84200F274
:105F6000CB8043462D1AA4B2B5FBF7F007FB1055C2
:105F700044EA05440EFB00FEA64508D91CEB0404C8
:105F800000F1FF3502D2A64500F2BB802846A4EB03
:105F90000E0440EA03409EE7C1F120078B4022FA3D
:105FA00007FC4CEA030C20FA07F405FA01F31C4342
:105FB000FD404FEA1C4900FA01F3B5FBF9F8200C4B
:105FC0001FFA8CFE09FB185540EA054508FB0EF048
:105FD000A84202FA01F20BD91CEB050508F1FF3AC1
:105FE00080F08880A84240F28580A8F102086544CC
:105FF0002D1AA4B2B5FBF9F009FB105544EA05458A
:1060000000FB0EFEAE4508D91CEB050500F1FF3480
:106010006CD2AE456AD90238654440EA0840A0FB1C
:106020000294A5EB0E05A542C846A64656D353D00A
:106030005EB1B3EB080265EB0E0505FA07F722FA2D
:1060400001F3CD401F43C6E900750021BDE8F0878C
:10605000C2F1200320FA03F10CFA02FC25FA03F343
:1060600095400D434FEA1C471FFA8CFEB3FBF7F136
:1060700007FB11302B0C43EA004301FB0EF0984262
:1060800004FA02F408D91CEB030301F1FF382FD204
:1060900098422DD9023963441B1AADB2B3FBF7F015
:1060A00007FB103345EA034500FB0EF3AB4208D96A
:1060B0001CEB050500F1FF3816D2AB4214D90238AB
:1060C0006544ED1A40EA014138E73146304607E7BA
:1060D0008646E5E61846FAE64B45A9D2B9EB020832
:1060E00064EB0C0E0138A3E74046EAE7204694E74C
:1060F0004146D1E7D0467BE7023B654432E708469C
:1061000009E76444023842E770B50D4D0D4C641B3D
:10611000A4100026A64209D10B4D0C4C00F020F82B
:10612000641BA4100026A64205D170BD55F8043B9F
:1061300098470136EEE755F8043B98470136F2E7F9
:10614000D0610008D0610008D0610008D461000867
:1061500002440346934200D1704703F8011BF9E75C
:10616000F8B500BFF8BC08BC9E467047F8B500BF44
:08617000F8BC08BC9E46704714
:10617800191B12131D1516171A090A0B1E0D0E0FDF
:1061880000000000000000000102030406070809DF
:10619800000000000102030402040608020C0810B3
:1061A80000000000000000000102030406070809BF
:1061B80054656B6B6F33322046342020000000009A
:0861C80070FCFF7F01000000E4
:0461D000C5160008E8
:0461D400A116000808
:1061D800007C000801010102701770177800640044
:1061E8006400D0070E004C046C07DC0564004A010B
:1061F800050A0A649001C800FF00CA0005011400DE
:106208004600DC05E803000010270000000000003D
:106218000A00000000000000640000000000000008
:10622800000000000000000000000000102700002F
:10623800FF0700000301060101010000D43000003F
:106248000105010AB400D007D0070000B400B70068
:10625800BA00BD00C100C400C700CA00CD00D0000C
:10626800D300D600D900DC00E000E300E600E90036
:10627800EC00EF00F200F500F700FA00FD00000165
:106288000301060109010B010E0111011301160199
:1062980019011B011E0120012301250128012A01E2
:1062A8002C012F0131013301350138013A013C013C
:1062B8003E014001420144014601470149014B01A9
:1062C8004D014E015001510153015401560157012E
:1062D80058015A015B015C015D015E015F016001CB
:1062E8006101620163016301640165016501660181
:1062F8006601670167016701680168016801680153
:106308006801680168016801680167016701670140
:10631800660166016501650164016301630162014B
:10632800610160015F015E015D015C015B015A0171
:1063380058015701560154015301510150014E01B2
:106348004D014B0149014701460144014201400109
:106358003E013C013A0138013501330131012F0179
:106368002C012A0128012501230120011E011B01FE
:1063780019011601130111010E010B010901060192
:1063880003010001FD00FA00F700F500F200EF003C
:10639800EC00E900E600E300E000DC00D900D600EC
:1063A800D300D000CD00CA00C700C400C100BD00A2
:1063B800BA00B700B400B100AE00AB00A700A4005B
:1063C800A1009E009B009800950092008F008C0011
:1063D8008800850082007F007C00790076007300C9
:1063E80071006E006B006800650062005F005D0070
:1063F8005A005700550052004F004D004A0048000F
:106408004500430040003E003C003900370035009D
:10641800330030002E002C002A002800260024001B
:10642800220021001F001D001B001A001800170081
:10643800150014001200110010000E000D000C00D1
:106448000B000A0009000800070006000500050007
:106458000400030003000200020001000100010023
:106468000000000000000000000000000000000024
:106478000000010001000100020002000300030007
:1064880004000500050006000700080009000A00CE
:106498000B000C000D000E0010001100120014007B
:1064A8001500170018001A001B001D001F0021000E
:1064B80022002400260028002A002C002E0030008C
:1064C80033003500370039003C003E0040004300EF
:1064D800450048004A004D004F0052005500570043
:1064E8005A005D005F006200650068006B006E0086
:1064F80071007300760079007C007F0082008500BF
:1065080088008C008F009200950098009B009E00E8
:10651800A100A400A700AB00AE00B10064001E03F8
:1065280003000000000000009001000000000000CF
:10653800E803000000000000000000000000000068
:1065480000000000204E0000A08601006419000031
:106558000000000001000000000000003200000000
:106568000000000000000000000000000000000023
:106578001027000050C30000010201006E00D00780
:1065880064000500E8030614320078004B005A0046
:106598005A001E0002010000FA000000204E2000F0
:0C65A80050C318070A00000000127A001F
:107BE00054454B4B4F33325F463431350000000073
:107BF0000000000000000000000000000000000085
:040000050800407936
:00000001FF
